:020000040000FA
:020000002F28A7
:08000800B1000308B2008312ED
:100010000B118613061386120612B009240830024B
:10002000031C8617331CB001331425083002031C4F
:10003000061726083002031C861627083002031C08
:100040000616B0090630B007051E33108518A30147
:100050000519A10132088300B10E310E0900831287
:1000600003138B01B3018312850107309F008316B0
:10007000FF308500831283169F010C1383128316B1
:10008000003086008312831681128B16811583122D
:100090000B118B17831286011E30A300FF30A400C2
:1000A000F121A401FF30A500F121A501FF30A60038
:1000B000F121A601FF30A700F121A701A30B4E28D3
:1000C0000030A400A500A6001E30A30002220222D8
:1000D0000222A40F6628FF30A400EB210222022294
:1000E000A40B0000A50F6E28A401FF30A500EB2192
:1000F00002220222A50B0000A60F7828A501FF30DE
:10010000A600EB2102220222A60B0000A70F8228E4
:10011000A601FF30A700EB2102220222A70B00005C
:10012000A40F8C28A701FF30A400A30B6B289828EC
:100130000030A400A500A6000730A3000222A40FEF
:100140009E28FF30A400E721E721F121FC21A40B28
:100150000000A50FA528A401FF30A500E721E72195
:10016000F121FC21A50B0000A60FB028A501FF304E
:10017000A600E721E721F121FC21A60B0000A70F33
:10018000BB28A601FF30A700E721E721F121FC21D0
:10019000A70B0000A40FC628A701FF30A400A30BE3
:1001A000A128D2280730A300FF30A400E721F121C5
:1001B000A401FF30A500E721F121A501FF30A60031
:1001C000E721F121A601FF30A700E721F121A701D6
:1001D000A30BD428EB280A30A300FF30A500A6000B
:1001E000A7008030A400F1214030A4002030A400FA
:1001F000F121A401EB21FF30A400A600A70080306C
:10020000A500F1214030A5002030A500F121A50175
:10021000EB21FF30A400A500A7008030A600F1214B
:100220004030A6002030A600F121A601EB21FF30CE
:10023000A400A500A6008030A700F1214030A7004F
:100240002030A700F121A701EB21A30BED280030FE
:10025000A400A500A6000A30A300FC21A40F2D29AC
:10026000FF30A400EB21FC21A50F3329FF30A500AE
:10027000EB21FC21A60F3929FF30A600EB21FC2140
:10028000A70F3F29FF30A700EB21FC21A40B452934
:100290000030A400EB21FC21A50B4B290030A50068
:1002A000EB21FC21A60B51290030A600EB21FC21FB
:1002B000A70B57290030A700F121A30B2D290730E8
:1002C000A300A401A501A601A70102220222022285
:1002D000A70F0000A40F6529FF30A400A700022289
:1002E000A40B0000A50F6F29FF30A500A401EB218E
:1002F0000222A50B0000A60F7829FF30A600A50159
:10030000EB210222A70B0000A40F8129FF30A400DB
:10031000A701EB210222A40B0000A50F8A29FF30C0
:10032000A500A401EB210222A50B0000A70F932931
:10033000FF30A700A501EB210222A60B0000A50FAC
:100340009C29FF30A500A601EB210222A70B00008B
:10035000A40FA529FF30A400A701EB210222A40BC2
:100360000000A60FAE29FF30A600A401EB21022257
:10037000A60B0000A70FB729FF30A700A601EB21AD
:100380000222A50B0000A40FC029FF30A400A50184
:10039000EB210222A70B0000A50FC929FF30A50001
:1003A000A701EB210222A50B0000A60FD229FF30E6
:1003B000A600A501EB210222A60B0000A70FDB2956
:1003C000FF30A700A601EB21A30B6F294C28EB21DE
:1003D000EB21EB210800F121F121F121F121F121A3
:1003E0000800FF30A100FF30A200A20BF529000099
:1003F000A10BF3290000080002220222022202229D
:10040000022208000230A100DC30A200A20B062A62
:0A0410000000A10B042A0000080000
:020FFE002F289A
:00000001FF
